:100000000C948D040C94AA040C94AA040C94AA04D5
:100010000C94AA040C94AA040C94AA040C94AA04A8
:100020000C94AA040C94AA040C940F0F0C94510E77
:100030000C94FC220C94AA040C94AA040C94AA0418
:100040000C94AA040C94AA040C94AA040C94AA0478
:100050000C94AA040C9419100C94AA040C94AA04ED
:100060000C94AA040C94AA040C94AA040C94AA0458
:100070000C94AA040C94AA040C94AA040C94AA0448
:100080000C94AA040C94AA040C94AA040C94AA0438
:100090000C94AA040C94AA040C94AA040C94AA0428
:1000A0000C94AA040C94AA040C94AA042C082C08FE
:1000B0005F085F08CA08E808F209F209F30867094F
:1000C00078097809640C8B0C390E8B0C390ED70C1F
:1000D000FA0C390EEF0DFF0D00201120DC1F7C20E3
:1000E0006C207A207A2078207A20CC25D125DB2537
:1000F000CF25D425D925D7258327862789278C275F
:100100008F279227952700000000000000000000C4
:1001100000000000000000000000000000000000DF
:10012000000000000000000000007E0F00D4FFFF70
:10013000FFC70000007800000000000000002A2B2C
:100140002800000000000000000000000000000087
:100150000029000000002C1E3420212224342627F0
:10016000252E362D3738271E1F2021222324252611
:100170003333362E37381F0405060708090A0B0CDF
:100180000D0E0F101112131415161718191A1B1C27
:100190001D2F3130232D350405060708090A0B0CE5
:1001A0000D0E0F101112131415161718191A1B1C07
:1001B0001D2F3130354C0102E00102E30101140131
:1001C00003E30103E00005010980A1018503190192
:1001D0002AB700150126B700950175108100C005EA
:1001E0000C0901A101850419012AA002150126A00C
:1001F00002950175108100C005010906A10185065F
:10020000050719E029E71500250195087501810208
:100210000507190029EF1500250195F075018102E8
:1002200005081901290595057501910295017503C8
:100230009101C005010902A1010901A100050919E7
:10024000012908150025019508750181020501099C
:100250003009311581257F95027508810609381509
:1002600081257F950175088106050C0A38021581E4
:10027000257F950175088106C0C00660FF0961A150
:10028000010962150026FF009520750881020963A7
:10029000150026FF00952075089102C0050109068A
:1002A000A101050719E029E7150025019508750149
:1002B00081029501750881010507190029FF1500C4
:1002C00026FF009506750881000508190129059586
:1002D0000575019102950175039101C00902740031
:1002E000040100A0FA090400000103010100092132
:1002F00011010001224000070581030800010904E3
:100300000100020300000009211101000122220066
:1003100007058303200001070504032000010904E9
:10032000020001030102000921110100012247001E
:10033000070582030800010904030001030000000F
:10034000092111010001226D00070585032000012C
:1003500012010002000000089732764901000102F4
:10036000000120034500720067006F0044006F0029
:100370007800200045005A00200047006C006F0004
:100380007700000028035A00530041002000540069
:100390006500630068006E006F006C006F0067000E
:1003A000790020004C00610062007300000004032B
:1003B000090429004C00E000E100025400001E0086
:1003C000140004001D0001534D001F001A00160008
:1003D0001B00E3052A002000080007000600E200D9
:1003E0002C002100150009001900E3004A0022003A
:1003F00017000A00050000004B005000E304000055
:10040000E00800004E004F00B75D0000E201000070
:10041000350023001C000B001100000034002400F4
:1004200018000D00100052002E0025000C000E00D8
:10043000360051002800260012000F0037002F0060
:100440002B00270013003300380030002D002D0052
:1004500031003400005CB65D0000010001000100C5
:100460000100010000000100010001000100010085
:10047000010001000100EF00010001000100010086
:10048000ED00EE000100F100010001000100F000AC
:100490000100F20001000100010001000100000064
:1004A0000100010001000000010000000100010046
:1004B0000100000001000000010001000100010036
:1004C0000100000001000100010001000100A9007D
:1004D0000100010001000100AC00AA00B60001000B
:1004E00001000100AB00A8000100010001000100B3
:1004F00001000100010001000100AE000100010047
:1005000000000100010001000100010000000100E5
:1005100001000100010001000100010001000100D3
:1005200001000100010001000100010001000100C3
:1005300001000100010001000100010001000100B3
:1005400001000100010000000100010001000000A5
:100550000100000001000100010000000100000096
:100560000100010001005000010000000100010035
:1005700001005200010001000100010001005100D2
:10058000010001000100010001004F000100010015
:100590000100010001000100010001000100010053
:1005A0000100010001000100000000443454007407
:1005B00064840055456500857595003626460066BD
:1005C0005676009686A6003727470077678700385B
:1005D0002848008878980039294900695979009994
:1005E00089A9003A2A4A006A5A7A003B2B4B006BD1
:1005F0005B7B004C3C5C007C6C8C005D4D6D008D29
:100600007D9D003E2E4E006E5E7E0144345401748A
:100610006484015545650185759501362646016658
:100620005676019686A601372747017767870138F6
:10063000284801887898013929490169597901992F
:1006400089A9013A2A4A016A5A7A013B2B4B016B6C
:100650005B7B014C3C5C017C6C8C015D4D6D018DC4
:100660007D9D013E2E4E016E5E7EBCFFFFBCFFFFF6
:10067000BCFFFFBCFFFFBCFFFFBCFFFFBCFFFFBC1C
:10068000FFFFBCFFFFBCFFFFBCFFFFBCFFFFBCFFC9
:10069000FFBCFFFFBCFFFFBCFFFFBCFFFFBCFFFFB9
:1006A000BCFFFFBCFFFFBCFFFFBCFFFFBCFFFFBCEC
:1006B000FFFFBCFFFFBCFFFFBCFFFFBCFFFFBCFF99
:1006C000FFBCFFFFBCFFFFBCFFFFBCFFFFBCFFFF89
:1006D000BCFFFFBCFFFFBCFFFFBCFFFFBCFFFFBCBC
:1006E000FFFFBCFFFFBCFFFFBCFFFFBCFFFFBCFF69
:1006F000FFBCFFFFBCFFFFBCFFFF00F5F500F5F5F9
:1007000000F5F500F5F500F5F500F5F500F5F50057
:10071000F5F500F5F500F5F500F5F500F5F500F552
:10072000F500F5F500F5F500F5F500F5F500F5F542
:1007300000F5F500F5F500F5F500F5F500F5F50027
:10074000F5F500F5F500F5F500F5F500F5F500F522
:10075000F500F5F500F5F500F5F500F5F500F5F512
:1007600000F5F500F5F500F5F500F5F500F5F500F7
:10077000F5F500F5F500F5F500F5F500F5F500F5F2
:10078000F500F5F500F5F500F5F583FFFF83FFFFB4
:1007900083FFFF83FFFF83FFFF83FFFF83FFFF8351
:1007A000FFFF83FFFF83FFFF83FFFF83FFFF83FFC5
:1007B000FF83FFFF83FFFF83FFFF83FFFF83FFFFB5
:1007C00083FFFF83FFFF83FFFF83FFFF83FFFF8321
:1007D000FFFF83FFFF83FFFF83FFFF83FFFF83FF95
:1007E000FF83FFFF83FFFF83FFFF83FFFF83FFFF85
:1007F00083FFFF83FFFF83FFFF83FFFF83FFFF83F1
:10080000FFFF83FFFF83FFFF83FFFF83FFFF83FF64
:10081000FF83FFFF83FFFF83FFFF00010101010151
:1008200001010101020202020202020202030303A9
:100830000303030303040404040404040505050579
:100840000506060606060707070707080808080939
:100850000909090A0A0A0B0B0B0C0C0C0D0D0D0EE5
:100860000E0E0F0F0F10101111111212131314147A
:10087000151516161717181819191A1A1B1B1C1DEF
:100880001D1E1E1F20202122222324242526262748
:100890002829292A2B2C2D2D2E2F3031323233347A
:1008A00035363738393A3B3C3D3E3F404142434480
:1008B00045464748494A4C4D4E4F50515354555662
:1008C00058595A5B5D5E5F616264656668696B6C0E
:1008D0006D6F7072737577787A7B7D7E8082838589
:1008E00087888A8C8E8F91939596989A9C9EA0A2C9
:1008F000A3A5A7A9ABADAFB1B3B5B7BABCBEC0C2D3
:10090000C4C6C9CBCDCFD1D4D6D8DBDDDFE2E4E796
:10091000E9EBEEF0F3F5F8FAFDFF11241FBECFEF7F
:10092000DAE0DEBFCDBF12E0A0E0B1E0E0E4FBE63C
:1009300002C005900D92A236B107D9F725E0A2E6D4
:10094000B2E001C01D92A23DB207E1F70E94B31CC4
:100950000C949E350C940000A5E2B0E0E2EBF4E0CC
:100960000C945931FC018081918123813481232BA6
:1009700031F09F3F31F491E08F3F19F403C091E0D3
:1009800001C090E090FD6CC57F0185E0DE0191968D
:1009900001900D928A95E1F7D70112962C9189A1C9
:1009A0009AA1222349F00E94272C182F682F89A191
:1009B0009AA10E94972C03C00E94632C182F69A152
:1009C0007AA1812F0E94CD168C019091C305F70169
:1009D0008281992309F44DC08111DCC2E091640247
:1009E000E330A0F481E08E0F80936402F0E0EE0F1C
:1009F000FF1FE85EFB4FD7018D919C91918380830F
:100A000082E08983CE0101960E94A52EBFEFE3ED1F
:100A1000F0E3B150E040F040E1F700C00000809109
:100A20006402833009F0B6C210926402EEE1F4E091
:100A3000A8E1B4E084E294E0318111962C91119701
:100A400032132EC030812C9132132AC03296129666
:100A50008E179F0789F784E0898381E08093C4051E
:100A60008EEF8A831092C305CE0101960E94A52EB7
:100A700091C29091C4059923C1F0882311F086E0BA
:100A800001C087E08983D7018C918A8311968C916C
:100A90008B838EEF8C83CE0101960E94A52E05C01C
:100AA00083E089831092C405DBCFF7018281033B89
:100AB000FDE51F07D1F5882309F43EC09091290474
:100AC00081E0890F8770987F853020F4892B80938F
:100AD000290402C090932904809129048770BFEFF4
:100AE0008B9FC0011124959587959595879599279A
:100AF000909389008093880090938B0080938A0064
:100B000090938D0080938C004091290450912A0489
:100B100060912B0470912C048FE090E00E94393298
:100B2000809128040E94B625C0C1043B2DE5120720
:100B300009F09EC08111B8C080916F0282720B3C97
:100B40009CE5190709F483C098F5063CBCE51B0732
:100B500009F469C0B8F4043CFCE51F0709F459C066
:100B600008F05CC0033C3CE5130709F025C29091F6
:100B7000C80581E089278093C805109220018091E3
:100B8000C70543C0083C9CE5190709F456C008F4A2
:100B90004FC0093CBCE51B0709F454C00A3CECE516
:100BA0001E0709F009C247E852E264E972E25DC03B
:100BB000003DFCE51F0709F473C098F40D3C3CE5CB
:100BC000130709F44EC008F447C00E3CACE51A0701
:100BD00009F464C00F3CBCE51B0709F0EDC185E0DA
:100BE00060C0073DECE51E0738F4023DFCE51F0739
:100BF00008F0D0C182E155C00F352DE5120709F488
:100C0000C9C1DAC19FEF9093CD0581608093C7057C
:100C1000C1C14FEC52E269ED72E227C049ED52E2E8
:100C20006FEC72E222C04BEB52E265EC72E21DC047
:100C300045EC52E26BEB72E218C041EA52E26EEA16
:100C400072E213C04EEA52E261EA72E20EC044E977
:100C500052E267E872E209C041EA50E26FEA70E2EC
:100C600004C04FEA50E261EA70E20E94972392C109
:100C7000033C3CE51307B9F1063BEDE51E0709F41B
:100C800047C0073BFDE51F0709F405C1053B2DE5FE
:100C9000120709F00AC1882309F47CC181E001C070
:100CA0008DE00E94622E76C18091290483FB222769
:100CB00020F991E0922790FB83F9809329049923EE
:100CC00029F040E060E080E00E94D41040912904C7
:100CD00050912A0460912B0470912C048FE090E0D5
:100CE0000E943932E2C0882309F454C19091CD05A5
:100CF0008091C7059F3F09F085CF1092CD05816097
:100D00008093C70540E060E080E00E94D41042C1BB
:100D1000882309F411CF26EBC22E21E0D22E3AE02F
:100D2000432EF6012491222309F4BFC0213009F09B
:100D30004EC031968491813069F4F2E0CF0ED11C1F
:100D4000F6018491893319F460E570E09CC060E09D
:100D500070E099C0823041F4F2E0CF0ED11CF60170
:100D600084910E94A52D93C0833041F4F2E0CF0E10
:100D7000D11CF60184910E94702D89C0843009F045
:100D800085C0F2E0CF0ED11CF601249180E090E006
:100D900030E0205331092A30310570F4489EA0011B
:100DA000499E500D1124C901840F951FFFEFCF1AE2
:100DB000DF0AF6012491ECCF009709F468C0AFE98F
:100DC000BFE01197F1F700C000000197F5CFE22FC7
:100DD000F0E0EA5CFE4F5490822F869586958695CA
:100DE00090E0FC01EA5DFE4F64902770712C022EAA
:100DF00002C0759467940A94E2F7B1E06B227724FD
:100E0000FC01EA5EFE4F8490912C022E02C0959464
:100E100087940A94E2F7E1E08E229924FC01EA5FCC
:100E2000FE4FA490B12C02C0B594A7942A95E2F786
:100E3000F1E0AF22BB246114710419F081EE0E942D
:100E4000A52D8114910409F402C386EE0E94A52DFC
:100E500029E3521609F4F5C260E070E0852D0E9486
:100E60004A2E8114910419F086EE0E94702D6114AF
:100E7000710419F081EE0E94702DA114B10439F0B3
:100E800060E070E08CE20E944A2E01C06F013FEFEB
:100E9000C31AD30A46CF882319F081E292E002C038
:100EA00080E090E00E944D2375C0D70112968C918E
:100EB000882309F441CE0C353DE5130709F464C0DD
:100EC00060F401159CE51907A9F00F3DACE51A0780
:100ED00009F072C00E9482184CC00E35BDE51B0798
:100EE00009F44AC008F452C0093AFDE51F0709F4A5
:100EF00040C062C010926F020E944B2D2FEF34E36E
:100F00008CE0215030408040E1F700C00000F894B0
:100F100081E08093E00080E28093D8001092C900C5
:100F2000AFE1BEE41197F1F700C000001DBA1092C6
:100F300068001CBC10BE1FBA10927A0010926E009E
:100F400010926F0010927100109272001092C900FE
:100F50001092BC0014B817B81AB81DB810BA109285
:100F6000BC0015B818B81BB81EB811BA0C94003FD5
:100F700011C00E949E250EC080916A0282FB8827C4
:100F800080F991E0892703C081E001C080E00E94E0
:100F9000771912C08091BB03877009F461C2F70111
:100FA0008281882309F45CC280916A0282FF58C260
:100FB00082E00E945A1954C2F70182810081118196
:100FC000882349F0C8010E94272CD82E682FC80119
:100FD0000E94972C04C0C8010E94632CD82EB8012F
:100FE0008D2D0E94CD160E94E616B82E192F982E30
:100FF000D70112960C9112971596AC90A2949FE08F
:10100000A9228091BB038770B9F00023A9F0812F3A
:10101000807F803421F080E28B0D883068F08091F1
:101020006A0282FF09C082E00E945A198091BB03C4
:101030008770DD24D3948111D12CC12EC2948FE00E
:10104000C8228C2D90E08C30910508F0CBC1FC01BA
:10105000EA5AFF4F0C946A34812F807F1F708823D7
:1010600011F01295107F0023B9F0112309F4A8C1E3
:1010700080E28B0D883010F0911006C080916F02D5
:10108000182B10936F0205C08091DC03182B10936E
:10109000DC030E94051994C18B2D0E94702D112331
:1010A00009F4A0C180E28B0D883080F1992071F1A4
:1010B00010958091DC0318231093DC032AC0812F44
:1010C000807F1F70803211F01295107F8B2D992038
:1010D00021F0B1E09B16D9F147C080916A0282FDF0
:1010E0001BC0002369F0112339F080916F02182B87
:1010F00010936F020E94051980E00E94A52D72C115
:1011000080E00E94702D112309F46CC1812F0E9490
:10111000FE180E94051966C1002381F08091DD034D
:10112000AA2051F0E1E0AE1207C0182B181709F4FD
:1011300059C11093DD0356C1812B10C0AA2021F0A4
:10114000F1E0AF1609F44EC10E94F8181FC0002349
:1011500041F021E02A1508F445C1812F0E94662D37
:1011600041C1A1103FC112C0002319F0AA20A9F368
:1011700027C1AA2059F0893309F031C13FEF87EE2A
:1011800093E0315080409040E1F727C1812F0E94C9
:101190005F2D28C1812F86958695837019F0813047
:1011A00061F020C1002321F08B2D912F937002C09C
:1011B00080E090E00E9463231BC1002321F08B2D6F
:1011C000912F937002C080E090E00E944D2310C1E7
:1011D0008B2D002319F00E94892B02C00E94CF2A78
:1011E0000E94E42B05C1812F8370A9F50111FEC077
:1011F0004B2D429546954770440F440F8B2D8F70B1
:1012000090E09C01042E01C0220F0A94EAF7B4FE7C
:1012100008C08FE090E001C0880F4A95EAF78095FA
:1012200001C080E0169516951370123069F088F4AD
:101230009091DE03113019F0822B892302C0922B8A
:10124000892B0E940F2DD2C0822B9091DE0389271B
:10125000F8CF822BF6CF002319F0812F817001C0C7
:101260008695882309F4C2C04B2D42954695477058
:10127000440F440F8B2D8F7090E09C01042E01C011
:10128000220F0A94EAF7B4FE08C08FE090E001C094
:10129000880F4A95EAF7809501C080E0169516956B
:1012A0001370123059F078F490912804113019F02D
:1012B000822B892309C0922B892B06C0822B909107
:1012C0002804892701C0822B0E94CC2C8FC01F705C
:1012D000002339F0812F0E94032D8B2D0E94662D53
:1012E00085C08B2D0E945F2D812F0E94F62C7EC021
:1012F0008B2DA2EF9A1669F1A91538F0B0EF9B1665
:1013000059F0E1EF9E1601F157C0F3EF9F1641F13E
:1013100024EF9216A9F050C0002369F0A11062C01A
:101320001F7181E090E001C0880F1A95EAF7909153
:10133000280489271FC031E03A1508F453C0F0CFC4
:1013400080916A0282FD19C0002329F0812F8F71DC
:1013500026C00023D9F3812F8F710E94F62C42C042
:10136000002339F01F7181E001C0880F1A95EAF758
:1013700001C080E00E94CC2C35C0002399F01F7181
:10138000812F0E94032D80916A0282FF07C0A8E08E
:101390001A9FC001112483608093BB03812F0E9498
:1013A000032D20C081E00E945A19B1E0BA15D0F493
:1013B00082E00E945A1916C0002321F0AA2031F2BF
:1013C0008B2D9BCEAA2039F2893349F4EFEFF7EE4B
:1013D00023E0E150F0402040E1F700C000008B2DF9
:1013E0000E94702D88EF8C0D843010F40E947923B8
:1013F000DD20B1F08091BB0380FD12C0D7011296B1
:101400001C928595859585950E94032DC7010E94A4
:10141000AC048091BB038595859585950E94F62C3B
:1014200085E0F701DE01119601900D928A95E1F7B2
:1014300009811A81C8010E94632CB8010E94CD164F
:101440000FC060E570E089E30E944A2E0DCDF9E3FC
:101450005F1202CD60E570E089E30E944A2E07CD5D
:10146000A596E0E10C9475318091950287FF11C03B
:101470008091E80082FD05C08091C6058111F8CFFA
:1014800011C08091E8008B770BC08091C60588233E
:1014900049F08091E80080FFF8CF8091E8008E77D6
:1014A0008093E8000895982F973068F59093E900AD
:1014B000981739F07091EC002091ED005091F000F8
:1014C00003C0242F762F50E021FD02C09F5FECCF98
:1014D0003091EB003E7F3093EB003091ED003D7F8B
:1014E0003093ED003091EB0031603093EB0070935E
:1014F000EC002093ED005093F0002091EE0027FDCA
:10150000E5CF80E008958F708093E90081E0089531
:1015100020919B0230919C022617370748F06115F5
:10152000710539F42091E8002E772093E80001C07E
:10153000B901FC0120E06115710579F18091C605C2
:101540008823F1F18530F1F18091E80083FD3CC002
:101550008091E80082FD2EC08091E80080FFEBCFF3
:101560002091F3008091F20090E0922B61157105BB
:1015700051F08830910538F421912093F1006150A9
:1015800071090196F3CF21E0089709F020E08091DE
:10159000E8008E778093E800CECF2111CFCF0AC02C
:1015A0008091C605882361F0853061F08091E80064
:1015B00083FD0AC08091E80082FFF2CF80E00895A9
:1015C00082E0089583E0089581E008950895809170
:1015D0007102089580936B0270936D0260936C02A8
:1015E0008091C605843001F585E08093E9008FEF96
:1015F0009091E800815095FD06C095ED9A95F1F720
:1016000000008111F5CF8091E80085FF0DC040E01A
:1016100050E063E070E08BE692E00E947B2E8091C8
:10162000E8008E778093E8000895BC0184E00E9472
:10163000EA0A0895BC0183E00E94EA0A089522E0C4
:101640002093E9002FEF3091E800215035FD06C0CE
:1016500035ED3A95F1F700002111F5CF2091E80022
:1016600025FF0BC040E050E065E070E00E947B2E5B
:101670008091E8008E778093E8000895CF93DF9300
:1016800020910A01222339F02091690227FF03C02B
:1016900060E225E002C068E021E02093E9002FEF3E
:1016A0003091E800215035FD06C035ED3A95F1F74F
:1016B00000002111F5CF2091E80025FF1DC0EC01AD
:1016C00080910A01811105C040E050E068E070E0BF
:1016D00003C070E040E050E0CE010E947B2E80917C
:1016E000E8008E778093E80080E2FE01A2E7B2E096
:1016F00001900D928A95E1F7DF91CF910895AAE2CA
:10170000B0E0E5E8FBE00C946631E5E9F2E08DE954
:1017100092E02091F10021938E179F07D1F78091DD
:101720009602833009F463C030F4813071F0823066
:1017300009F49FC0B6C08A3009F48BC08B3009F41D
:101740006EC0893009F0ADC020C080919502813A09
:1017500009F0A7C08091E800877F8093E80080911E
:10176000990290919A02892B21F460E282E792E03B
:1017700003C060E080E090E070E00E94880A809101
:10178000E8008B778093E8008CC0809195028132CD
:1017900009F087C08091990290919A02009719F000
:1017A000039709F07EC08091E800877F8093E8006E
:1017B0008091E80082FD05C08091C6058111F8CFB7
:1017C00070C02091F3008091F20090E0922B02977C
:1017D00031F48091F100813011F0863021F4809154
:1017E000F100809371028091E8008B7756C0809160
:1017F0009502813A09F055C08091990290919A0220
:10180000892B09F04EC08091E800877F8093E80023
:101810008091E80080FFFCCF80910A0139C080915F
:1018200095028132F1F58091990290919A02892B6B
:10183000C1F58091E800877F8093E8000E94340A18
:101840008091970280930A0110926F020E944B2DA3
:1018500028C080919502813221F58091E800877F30
:101860008093E8000E94340A80919802809370026D
:1018700018C080919502813AA1F48091E800877F99
:101880008093E8008091E80080FFFCCF8091700297
:101890008093F1008091E8008E778093E8000E94A9
:1018A000340A8091E80083FFE4C180919502909111
:1018B0009602492F50E04A30510508F0DAC1FA018A
:1018C000EE59FF4F0C946A34803821F0823809F0C9
:1018D000D0C108C08091920290919302992389F01F
:1018E00082600FC0809199028F70873008F0C1C16B
:1018F0008093E9008091EB0085FB882780F91092A6
:10190000E9009091E800977F9093E8008093F100C0
:101910001092F10070C1282F2D7F09F0AAC18823F1
:1019200019F0823061F0A5C180919702813009F0F1
:10193000A0C1933009F080E0809393022EC0809183
:10194000970281112AC0809199028F702FEF280F82
:10195000263008F08EC18093E9002091EB0020FF33
:101960001CC0933021F48091EB00806214C09091F0
:10197000EB0090619093EB0021E030E0A90102C000
:10198000440F551F8A95E2F74093EA001092EA004F
:101990008091EB0088608093EB001092E9008091C9
:1019A000E800877F8093E8000E94340A62C18111B9
:1019B00060C1109197021F778091E3008078812B9E
:1019C0008093E3008091E800877F8093E8000E9485
:1019D000340A8091E80080FFFCCF8091E3008068AA
:1019E0008093E300111102C082E001C083E0809384
:1019F000C6053FC18058823008F03BC12091970254
:101A0000309198022C3D53E0350779F583E08A83C5
:101A10008AE289834FB7F894DE01139620E03EE016
:101A200051E2E32FF0E050935700E49120FF03C010
:101A3000E295EF703F5FEF708E2F90E0EA3010F08C
:101A4000C79601C0C0968D939D932F5F243149F7AF
:101A50004FBF8091E800877F8093E8006AE270E0E2
:101A6000CE0101960E94880AB4C08091990290919B
:101A70009A02432F552743305105A9F068F44130AD
:101A8000510509F405C14230510509F0F2C084E75F
:101A900090E0ECEDF2E04BC04132510529F14232C9
:101AA000510589F1E6C0C901992781309105A1F05E
:101AB00058F0029709F0DDC0E2E6F3E0E4918E2FE2
:101AC00090E0E2E6F3E030C0EEEAF3E0E4918E2F3E
:101AD00090E0EEEAF3E028C0E4E8F3E0E4918E2F32
:101AE00090E0E4E8F3E020C08430910508F0C1C044
:101AF000880F991FFC01E05DFE4F0190F081E02D01
:101B000089E090E014C08430910508F0B2C0FC0177
:101B1000EE0FFF1FE85DFE4F0190F081E02DDC012C
:101B2000AC5DBE4F8C9190E0009709F4A2C020916B
:101B3000E800277F2093E80020919B0230919C02CF
:101B40002817390708F4C90140E0009789F120916E
:101B5000C605222309F43DC02530D9F12091E800C3
:101B600023FD37C02091E80022FD2FC02091E8001E
:101B700020FFEBCF4091F3002091F20030E0342BB6
:101B8000009759F02830310540F444914093F1001A
:101B9000319601972F5F3F4FF3CF41E02830310559
:101BA00009F040E02091E8002E772093E800CDCFA7
:101BB0004111CDCF0AC08091C605882351F08530F0
:101BC00041F08091E80083FD04C08091E80082FF2D
:101BD000F2CF8091E8008B778093E8004AC080388C
:101BE00009F047C08091E800877F8093E8008091EA
:101BF00094028093F1008091E8008E77D3CE81111A
:101C000038C08091970290919802992702978CF59D
:101C10008091E800877F8093E800109197021093ED
:101C200094020E94340A111106C08091E30087FDDE
:101C300002C081E001C084E08093C60542E061EC0F
:101C400081E00E94530A42E061EC82E00E94530A64
:101C500042E261EC85E00E94530A42E261EC83E0DB
:101C60000E94530A42E260EC84E00E94530A809191
:101C7000C6058091E80083FF10C08091E800877F4F
:101C80008093E8008091EB0080628093EB0005C0B8
:101C900082E190E0E0E5F3E04ACFAA96E3E00C941D
:101CA00082311F920F920FB60F9211242F933F9300
:101CB0004F935F936F937F938F939F93AF93BF9354
:101CC000CF93DF93EF93FF93C091E900CF708091A2
:101CD000EC00D82FD17080FDD0E81092E9008091FF
:101CE000F000877F8093F00078940E947F0B109221
:101CF000E9008091F00088608093F000CD2BCF70D8
:101D0000C093E900FF91EF91DF91CF91BF91AF9127
:101D10009F918F917F916F915F914F913F912F9103
:101D20000F900FBE0F901F901895E8EDF0E08081A6
:101D30008E7F80831092E2001092DA001092E10010
:101D4000A0EEB0E08C9181608C9380818F7780834E
:101D500019BCA7EDB0E08C918E7F8C9380818F7E33
:101D6000808310926E020895A0E0B0E0EAEBFEE0FE
:101D70000C946131C8EDD0E088818F7E8883E7EDD7
:101D8000F0E080818160808384E082BF81E0809385
:101D90006E0288818E7F888302EE10E0F801108247
:101DA0001092DA0081EEC82ED12CF60110828881C3
:101DB0008F77888388818068888388818F7D8883F6
:101DC00019BC1092C60510929402109293021092C0
:101DD000920290EEE92EF12CF70180818B7F8083B7
:101DE00088818160888342E060E080E00E94530A3D
:101DF000F60180818E7F8083F801808181608083FD
:101E0000808188608083F70180818E7F80838881D4
:101E100080618883CDB7DEB7E8E00C947D311F92F6
:101E20000F920FB60F9211242F933F934F935F930E
:101E30006F937F938F939F93AF93BF93EF93FF9392
:101E40008091E10082FF09C08091E20082FF05C01D
:101E50008091E1008B7F8093E1008091DA0080FF28
:101E60002AC08091D80080FF26C08091DA008E7F42
:101E70008093DA008091D90080FF18C080E189BD8D
:101E800082E189BD09B400FEFDCF81E08093C605E3
:101E900080916E0281110FC00E94950E0E94B40EB7
:101EA0008091E20084608093E20005C019BC10922A
:101EB000C60510926E028091E10080FF17C08091EC
:101EC000E20080FF13C08091E2008E7F8093E200E9
:101ED0008091E20080618093E2008091D80080626E
:101EE0008093D80019BC85E08093C6058091E100FD
:101EF00084FF30C08091E20084FF2CC080E189BD66
:101F000082E189BD09B400FEFDCF8091D8008F7DAC
:101F10008093D8008091E1008F7E8093E1008091D2
:101F2000E2008F7E8093E2008091E20081608093E6
:101F3000E20080919402882311F084E007C0809130
:101F4000E30087FD02C081E001C083E08093C60505
:101F50008091C6058091E10083FF27C08091E20057
:101F600083FF23C08091E100877F8093E10082E0BE
:101F70008093C605109294028091E1008E7F809339
:101F8000E1008091E2008E7F8093E2008091E20088
:101F900080618093E20042E060E080E00E94530AAA
:101FA0008091F00088608093F000FF91EF91BF91E5
:101FB000AF919F918F917F916F915F914F913F91E1
:101FC0002F910F900FBE0F901F9018952091E40055
:101FD0003091E50095E64091EC00842F817040FF40
:101FE00023C08091E80080FD1DC08091C605882334
:101FF00099F0853099F08091EB0085FD11C04091FA
:10200000E4005091E5002417350729F3915011F0B1
:102010009A01E1CF84E0089582E0089583E0089575
:1020200081E0089580E008954091E80042FFDDCF0F
:10203000089578941F920F920FB60F9211248F93E8
:102040009F93AF93BF938091650290916602A09198
:102050006702B09168020196A11DB11D80936502CF
:1020600090936602A0936702B0936802BF91AF910C
:102070009F918F910F900FBE0F901F9018959C010C
:102080004FB7F8948091650290916602A091670223
:10209000B09168024FBF821B930B0895E42FF0E0CC
:1020A000EE0FFF1FEF52FE4F9081921B97FD91950F
:1020B000292F38E1239F212D1124620F08950F93BA
:1020C0001F9310E0F801EE0FFF1FEF52FE4F9081BB
:1020D000905797FD9195000F111FF801EE52FE4F9A
:1020E000E081F0E0B097DF01AA0FBB1F8D010E0F5A
:1020F0001F1F2003D001219FB00D1124E8E3F0E061
:10210000E91BF10997FDF3959F01220F331F890108
:102110000E0F1F1F40039001419F300D11242A0F05
:102120003B1F37FF02C021583F4F220F232F221F92
:10213000330B620F1F910F9108952091CC0530E170
:10214000230F08F42FEF60E1822F90E00E943B2ADA
:10215000BC0188EB9BE00E94433180E090E0089551
:102160000F931F93CF93DF93D62F072F182FC42FD2
:10217000822F0E94AB29EC2FF0E0EE0FFF1FEF52F1
:10218000FE4F90819058890F87FD8195880F682FA9
:102190002CE0629F612D11246D0F702F812FDF9134
:1021A000CF911F910F9108950E94FB2008950E94E6
:1021B000BD200895A4E0B0E0E0EEF0E10C945831C9
:1021C000782E80911A0187110DC02091C8052370C7
:1021D00030E04091190150E081E02417350719F4EF
:1021E00080E001C081E0817080931F018091CD0566
:1021F00090911E01981739F080931E0140E060E035
:1022000080E00E94D410EFE07E125DC08BE598E282
:102210000E94D12E8A8342C0F71508F49AC123E0A8
:10222000721609F459C0271508F4F7C031E0731687
:1022300009F497C0371508F0B6C080911D01382FFA
:10224000330F330F380F398375E0F72EF30E80E329
:102250008F1510F460E3F62E1091CA059091CB050E
:102260009A830091C905B801892F0E94452AE62E5C
:10227000D72EC82E6091CC05600F712F8A810E94E5
:10228000452A6A83172F082F29812F1508F4ABC020
:1022900031E03A838FE28F1508F48EC080911D01E2
:1022A0008F5F80931D019A81911113C582E0809305
:1022B000200180911F0181110CC571100AC583E0B6
:1022C0008093200106C5E71508F46BC1F7E07F1283
:1022D000A3CF8AE898E29CCF80911D01982F990F97
:1022E000990F980F99839B5F9B83913310F0E0E3E4
:1022F000EB83E090CA05D090CB052091CC0550E44B
:10230000F52E3F2D329F312D1124F32EE981FB81D3
:10231000EF1708F042C08981082F10E0F801EF5C48
:10232000FD4F908180911E018923B9F0F801EE0FD5
:10233000FF1FEE52FE4F808182958F706091C9051C
:102340008F9D600D11247E2D8D2D0E94452A462FD4
:10235000282F672FC8010E94D71099819F5F99830A
:10236000D5CF80911D01282F220F220F280F2983FE
:102370002B5F2B83213310F030E33B836091C90541
:102380007091CA058091CB050E94452A162F072F10
:10239000F82EE981FB81EF1788F021E02A83F033E2
:1023A00008F47CCF09C080911F01882329F040E008
:1023B00060E080E00E94D4101A8270CF8981E82FFB
:1023C000F0E0DF01AF5CBD4F8C9190911E0198232E
:1023D00031F02F2D412F602FCF010E94D71099810E
:1023E0009F5F9983D6CFE9818E2F90E0FC01EF5C4F
:1023F000FD4F308120911E01232359F030FF04C08E
:10240000202F4A81612F03C02C2D4E2D6D2D0E944F
:10241000D710F981FF5FF98337CF85E078124AC082
:1024200080911D01382F330F330F380F39833B5FF5
:102430003B83313310F080E38B830091C905109109
:10244000CA05F090CB056091CC05669566956695BA
:102450008091BF059091C0050E943B2A0E94AB2944
:10246000805887FD8195880F282F3F2D239F212D90
:102470001124822FB8010E94452A162F072FF82E0B
:10248000E981FB81EF1708F088CF8981E82FF0E020
:10249000DF01AF5CBD4F8C9190911E01982331F00C
:1024A0002F2D412F602FCF010E94D71099819F5F60
:1024B0009983E6CF871508F449C080911D01382F14
:1024C000330F330F380F39833B5F3B83313310F0C9
:1024D00080E38B83E090CA05D090CB052091CC059A
:1024E00030E4F32E3F2D329F312D1124F32EE9815C
:1024F000FB81EF1708F051CF8981082F10E0F80118
:10250000EF5CFD4F908180911E018923D9F0F80185
:10251000EE0FFF1FEF52FE4F6081F69EB0011124B7
:1025200025E0759567952A95E1F78091C905680FB3
:102530007E2D8D2D0E94452A462F282F672FC801FA
:102540000E94D71099819F5F9983D1CF86EB98E243
:102550005FCE9BE0791208C089E399E202C085E56D
:1025600099E20E94702F56CE971568F0E9E07E122E
:1025700005C080E799E20E94EC2F4CCEE71578F376
:102580008EE899E2F8CFFDE07F1203C08FE798E272
:102590003FCEF71518F088E898E23ACE86E798E241
:1025A00037CE27E172124FC080911D01382F330FB3
:1025B000330F380F3983132F1B5F113308F010E3EB
:1025C00080911F0181111EC06091CC0520E1620F36
:1025D00008F46FEF8091BF059091C0050E943B2ADF
:1025E0006AE070E00E944331892B21F50E94CC29DA
:1025F00060E30E944A3460911E01892F90E00E949E
:10260000C22318C09981892F90E09C838B83E12E8F
:10261000F12C2B813C812E153F0564F460911E0145
:102620008B819C810E94C223EB81FC813196FC83CB
:10263000EB83EFCF31E03A8302C091E09A8310330D
:1026400008F42CCEB9CE271530F133E1731203C054
:1026500084E199E286CF371570F081E1781203C0EA
:1026600082E19AE288CF871518F08CE498E279CF5E
:1026700088E299E280CF95E1791203C08CEE97E26F
:1026800004C0971528F08EE198E20E941B2FC2CD5E
:102690008FE590E1FACFEBE17E1203C08EE490E18A
:1026A000B7CDE71508F4A1C0F9E17F1250C08091C1
:1026B0001D01E82FEE0FEE0FE80FE983EB5FEB83D0
:1026C000E13310F0F0E3FB830091CA051091CB05D4
:1026D000F090C9056091CC056695669566958091E8
:1026E000BF059091C0050E943B2A0E94AB298058EB
:1026F00087FD8195880F682F2CE0629F612D112442
:102700006F0D702F812F0E94452A162F072FF82E4C
:1027100089819B818917A8F42981E22FF0E0DF01EC
:10272000AF5CBD4F8C9190911E01982331F02F2DFD
:10273000412F602FCF010E94D71039813F5F39832D
:10274000E7CFE1E0EA83903308F4A8CD35CEF71562
:1027500008F448C080911F0181111EC06091CC0512
:1027600020E1620F08F46FEF8091BF059091C005E2
:102770000E943B2A65E070E00E944331892B09F0FA
:102780001BCE0E94DA3160E370E00E945634609103
:102790001E010E949E2310CE80911D01982F990F3B
:1027A000990F980F9983192F1B5F113308F010E3CD
:1027B000F981EF2FF0E0FC83EB83E12EF12C8B818C
:1027C0009C818E159F050CF038CF60911E018B8186
:1027D0009C810E949E232B813C812F5F3F4F3C8335
:1027E0002B83EDCF80EB90E113CD2DE17212F0C081
:1027F000409131035091320360913303709134035F
:102800008091BF059091C005A091C105B091C2050E
:1028100084179507A607B70708F4CECD80911F014E
:1028200081110EC080911D01982F990F990F980F5B
:102830009983092F0B5F013308F45CC000E35AC091
:1028400040E060E080E00E94D41001EA12E01C82C7
:102850001B828FE7D82E0E94CC2981FF05C0F8018A
:1028600010821182128220C00E94CC29C82E0E94A0
:10287000CC298695782F2D2D720F08F47FEF8B8150
:102880009C81880F991FEB81FC818E0F9F1F9C01FB
:102890002F553D4F79016C2D8091CB050E94452A23
:1028A000F7016083718382832B813C812F5F3F4FCF
:1028B0003C832B830D5F1F4F2033310561F6B2CF70
:1028C0003981832F90E0FC01EF5CFD4F3081209136
:1028D0001E01232361F0FC01EE0FFF1FE80FF91F1B
:1028E000EF55FD4F2281408161810E94D71089817F
:1028F0008F5F89839981901718F3E1E0EA830033B1
:1029000008F01A82003308F4C9CC20E010E001502E
:102910001109822F90E080179107CCF4AC01440F8D
:10292000551F480F591F4F555D4F0196FC01EE0F83
:10293000FF1F8E0F9F1FFC01EF55FD4F808191817E
:10294000A281FA0180839183A2832F5FE2CF0E944C
:10295000CC297801EE0CFF1C81FF09C00E0D1F1D54
:10296000F801EF55FD4F10821182128218C00E94AB
:10297000CC2989830E94CC298695782F2FE7720F66
:1029800008F47FEF0E0D1F1D0F551D4F69818091BB
:10299000CB050E94452AF8016083718382830E94DF
:1029A0009D100091BF051091C0052091C105309187
:1029B000C205DC01CB01800F911FA21FB31F8093C2
:1029C000310390933203A0933303B093340366CC66
:1029D000721608F07AC080911D01982F990F990FF7
:1029E000890F8B5F8B834091BF055091C00560912B
:1029F000C1057091C20580919D0290919E02A091A7
:102A00009F02B091A00284179507A607B70708F0A8
:102A100055C00E94CC2989830E94CC2990E3891B50
:102A2000F0F7890F082F10E0F801EF5CFD4F80915F
:102A30001E019081982309F441C0F981F1FF04C07F
:102A400020E040E060E013C00E94CC2989830E940E
:102A5000CC298695782F2FE7720F08F47FEF6981D4
:102A60008091CB050E94452A462F282F672FC80149
:102A70000E94D7102091CC0530E1230F08F42FEFEE
:102A800060E1822F90E00E943B2ABC0184EF91E03C
:102A90000E9443318091BF059091C005A091C1056E
:102AA000B091C205860F971FA11DB11D80939D0295
:102AB00090939E02A0939F02B093A00221E02A83EC
:102AC0003B81303308F4EACB77CC3EE17312C7C0C8
:102AD00080911F01882329F040E060E080E00E949F
:102AE000D41080911D01982F990F990F890F8B5F3A
:102AF00089834091BF055091C0056091C1057091D7
:102B0000C20580915F0390916003A0916103B09131
:102B1000620384179507A607B70708F099C060916C
:102B2000C9057091CA058091CB050E94452A662E81
:102B3000572E482E05E313E02DE731E03C832B832D
:102B400041ED842E41E0942EAB80BC80650178017C
:102B500032E0332EF7018081F601882369F080810D
:102B6000242D462D652D90E00E94D710F50185811A
:102B7000242D462D652D0CC0808120E040E060E0D2
:102B800090E00E94D710F501858120E040E060E0F0
:102B900090E00E94D710F701818181937F013A94E0
:102BA000FFEFCF1ADF0A21E0A21AB1083110D2CF0D
:102BB000F8018281EB81FC81882371F08281242DD0
:102BC000462D652D90E00E94D710EB81FC8183811A
:102BD000242D462D652D0DC0828120E040E060E06F
:102BE00090E00E94D710EB81FC81838120E040E0DF
:102BF00060E090E00E94D7100E94CC29837091E0A1
:102C000009F090E0F80192830D5F1F4F2B813C810A
:102C10002A5F3F4F3C832B838216930609F094CFA3
:102C20000E949D100091BF051091C0052091C10523
:102C30003091C205DC01CB01800F911FA21FB31F91
:102C400080935F0390936003A0936103B09362034A
:102C500031E03A838981803308F420CBADCB8FEF0C
:102C6000781231C08091BF059091C005A091C10537
:102C7000B091C20588279C70AA27BB272AE0B69589
:102C8000A795979587952A95D1F782309105A1054B
:102C9000B10571F083309105A105B10569F040E0FF
:102CA0000197A105B10511F060E008C064E102C020
:102CB00044E160E080E003C044E164E184E10E941B
:102CC000D41082E0FDCA80911D018F5F80931D01A9
:102CD000EDCA2496E1E10C947431E8ECF5E085E36B
:102CE00080838091210190912201A0912301818311
:102CF0009283A3838CE384838FEF858346E050E047
:102D00006CE170E0CF010E9417321092C705089560
:102D100080E008959091690292FF0DC0282F2871DC
:102D2000283019F4877F846006C0282F247124304E
:102D300011F48B7F886093FF0DC0282F28712831F4
:102D400019F4877E846106C0282F2471243111F480
:102D50008B7E886120916A0220FF0DC0382F387168
:102D6000383019F4877F816006C0382F31713130D7
:102D700011F48E7F886021FF0DC0282F2871283123
:102D800019F4877E816106C0282F2171213111F449
:102D90008E7E886194FD877E08957E30A0F4663033
:102DA00090F494E5899FF001112486E0789FE00D6E
:102DB000F11D1124E60FF11DEE0FFF1FEE54FC4F25
:102DC00085919491089580E090E00895CF93DF93EA
:102DD0008238910569F1B0F48133910509F477C027
:102DE00048F48932910509F469C08A32910509F4E1
:102DF00073C092C08533910509F45BC08933910596
:102E0000B9F08AC0833E910591F138F4803E910576
:102E1000D1F0823E910531F17FC0863E9105D9F116
:102E2000873E9105E9F1843E910509F075C028C0FF
:102E30002091690220FD5BC021FD59C020916A02EA
:102E400023FD61C069C08091690280FD4AC0809104
:102E50006A0280FF4CC08091690284FD4EC183EEFE
:102E600090E04DC18091690282FF3EC0F4CF809115
:102E7000690282FD39C080916A0280FD38C0EBCFC3
:102E800080916A0281FF39C08091690284FD35C159
:102E900087EE90E034C18091690283FF2BC0F4CFAC
:102EA0008091690283FD26C080916A0281FD25C060
:102EB000EBCF8091690285FD26C022C08091690216
:102EC00085FD1EC080916A0283FF1DC00AC08091EB
:102ED000690286FD1BC01DC08091690286FD19C074
:102EE00015C089E390E00BC182EE90E008C180EE4E
:102EF00090E005C186EE90E002C184EE90E0FFC054
:102F000085E390E0FCC089E290E0F9C08AE290E0BD
:102F1000F6C081E390E0F3C0811531E5930708F036
:102F200061C0811520E59207B0F09C012370332722
:102F300041E050E002C0440F551F2A95E2F7282FC8
:102F40002695269580E2289F90011124CA01822BA4
:102F5000932B9D68D4C0883E910568F5803E91050D
:102F600008F0CDC0883A9105B8F4853A910548F04B
:102F7000855AE82FF0E0E85CFE4F808190E0906495
:102F8000BEC08130910509F4B5C008F4B6C08430E4
:102F9000910508F4B2C0B3C08F3B910508F0ADC0F5
:102FA000885AE82FF0E0EE0FFF1FE55CFE4F8081AE
:102FB00091819464A4C0811530E2930758F481157F
:102FC00021E0920708F09BC08D3E910508F495C062
:102FD000906595C0811530E4930708F48EC09F700A
:102FE000906A8DC0811525E5920708F042C08115D1
:102FF00034E5930728F0982F8827846F906A7FC064
:10300000811523E59207B0F09C012370332741E03E
:1030100050E002C0440F551F2A95E2F7282F26954D
:10302000269580E2289F90011124CA01822B932BC0
:103030009A6865C0811532E5930728F4982F882790
:10304000816F906A5CC09C012370332741E050E09F
:1030500002C0440F551F2A95E2F7282F2695269582
:1030600080E2289F90011124CA01822B932B9C6837
:1030700046C0EC01C11589E5D807B0F4C11528E5B3
:10308000D20728F09C2F8827806F906A38C0C1151E
:1030900036E5D30790F58C2F0E948A168F7190E049
:1030A000982F882790622BC0C1158AE5D80790F425
:1030B0008C2F8F700E948A1694E0D695C7959A95AA
:1030C000E1F7CF70D0E0DC2FCC27D0699E01282B10
:1030D000C90115C0CE0190568115904270F48D2F14
:1030E0008F710E948A16282F2F71CE019927906226
:1030F000922B05C081E090E002C080E090E0DF917B
:10310000CF91089568EE7EEF80E090E00E94453216
:1031100060E082E090E00E94273260E083E090E08F
:103120000E9427321092DE0360E084E090E00E946B
:10313000273264E082E290E00E94273260E085E07E
:1031400090E00E94273260E086E090E00E94273203
:103150006FEF87E090E00E94273240E050E0BA0134
:1031600088E090E00E94393260E08DE090E00E94BB
:10317000273240E050E0BA0188E190E00E94393205
:1031800060E087E190E00E94273240E050E0BA0121
:103190008CE190E00E94393260E070E080E290E0E3
:1031A0000E94453240E050E0BA0188E190E00E9480
:1031B00039321092290410922A0410922B04109292
:1031C0002C0484E0809329044091290450912A041E
:1031D00060912B0470912C048FE090E00E943932B2
:1031E00040E050E0BA0183E190E00E943932089556
:1031F0008091DD0381111092DD03089580959091F7
:103200006F02892380936F02089590916F028091DD
:10321000DC03982B909363038091DD038823D9F01E
:10322000892B8093630380910A01882331F0809178
:10323000690287FF02C08EE101C086E0E5E6F3E0A7
:1032400090E0815028F021912223D9F39F5FF9CF9C
:1032500091110E94F81840E250E06CEB73E083E6B5
:1032600093E00E949135892B21F180E2E3E6F3E0BF
:10327000ACEBB3E001900D928A95E1F7E0918C05FB
:10328000F0918D053097A9F080910A01882359F0BB
:103290008091690287FF07C0809163038093640374
:1032A00086E0809363030280F381E02D83E693E060
:1032B000099508952091BB03809582238093BB03D9
:1032C000982F977099F430E0482F082E000C550B7A
:1032D0002417350759F090916A0292FF07C085952F
:1032E000859585950E94F62C1092BB030895CF9387
:1032F000C0916A02C2FB992790F9981791F080FB60
:10330000C2F9C0936A026091690284E090E00E9471
:1033100027326C2F82E290E00E94273282E00E94E6
:103320005A19CF9108958091BA0390918903891712
:1033300019F08F5F8770FBCF08950F931F93CF9382
:10334000DF938091880382958F7009F05AC0809135
:103350008503882309F455C08091BA03109189032D
:103360006091830370918403C0918603D091870399
:1033700091E06F3F09F090E0292F06E0811709F4F2
:1033800040C0209721F07F3F21F030E003C031E0C2
:1033900001C0322F90E030FD31C0089FF001099F3D
:1033A000F00D1124DF01A657BC4F11963C911197E7
:1033B000371324C03C91361321C012963C911297CA
:1033C00031111CC013964D915C9114974C1B5D0BF1
:1033D000483C510598F4809188038F7080618093F8
:1033E0008803E157FC4F80818F708061808383E880
:1033F00093E00E94AC040E94931903C00196877069
:10340000BDCFDF91CF911F910F910895A1E1B0E061
:10341000ECE0FAE10C945E318C0185E0F801DE010C
:103420001D9601900D928A95E1F7F801E280909146
:103430008303609184034091860350918703411573
:10344000510531F06F3F31F481E09F3F19F403C023
:1034500081E001C080E0F82FF1709F2E80FD1BC13C
:10346000F80130812181C380D48083E8A82E83E0D5
:10347000B82EF0908503F601E41BF50BFF2009F44C
:10348000C7C080918803E83CF10508F092C0482F3E
:10349000407F09F051C0621311C093130FC0FE2C7E
:1034A000E1100CC08F70806180938803C5010E9479
:1034B000AC0480918803F80185832AC1C114D1042A
:1034C00031F02F3F31F481E03F3F19F403C081E038
:1034D00001C080E080FD03C081E08E2502C080E055
:1034E00090E0F82FF170FF2E80FF1CC08091BA038E
:1034F0004091890356E0841709F4E8C090E0589F92
:10350000F001599FF00D1124E657FC4F61812613FD
:1035100006C06081631303C06281E61203C0019696
:103520008770E9CFFE2CEE2009F4F2C08091880369
:1035300081608093880349C0621306C0931304C05E
:10354000E11002C0F80186C0C8010E94142D882332
:1035500051F1EE2041F120918803822F82958F70E6
:1035600090E0029774F08091830390918403988790
:103570008F831986DB86CA862C87CE0107960E9428
:10358000AC0486E0F801A3E8B3E001900D928A95BF
:10359000E1F70E949D190AC06217C9F0C8010E9494
:1035A000142D81111EC0C8010E94AC04FF24F394A5
:1035B000AFC0482F407F81F783E893E00E94AC04BE
:1035C00086E0F50111928A95E9F7F12CA1C09313D9
:1035D000E5CFE110E3CFF8018583C8010E94AC0478
:1035E00054C0EE2001F320918803822F82958F70C2
:1035F00090E0029734F280918303909184039A8340
:1036000089831B82DD82CC822E83CE010196B7CFC7
:10361000E83CF105D0F5FE2CEE2029F2621327C01C
:10362000931325C02091880320FD18C0822F829516
:103630008F70482F50E04115510581F0F801258326
:103640004F30510541F08F5F982F9295907F822FD8
:103650008F70892B8583C8010E94AC0486E0F80135
:10366000A3E8B3E001900D928A95E1F751C0C8013B
:103670000E94142D811185CF8091880381608093F1
:103680008803C8010E94AC0443C086E0F501119292
:103690008A95E9F73DC0EE2009F485CFC8010E9464
:1036A000142DF82E882309F47ECF86E0F801A3E8D4
:1036B000B3E001900D928A95E1F780918303909198
:1036C00084030E94562C0E949D1922C03D872E879C
:1036D0008D859E850E94562C292F22952F70223091
:1036E00028F49F7039F0811105C00BC0243028F4F4
:1036F0009F7049F4805E883020F0C8010E94AC04BD
:103700009F2CF92C05C0F8019581907F99F7F9CF8E
:103710008F2D6196EBE00C947A31A0E0B0E0E3E904
:10372000FBE10C9461318091170190911801892B74
:10373000A1F08091DF038F5F8093DF0381110DC0C3
:103740000E945E2690E09093180180931701892BC8
:1037500021F40E94D5260E940A240AEE13E0780183
:10376000D0E0C0E087E0C82ECC0E8C2F0E94452709
:103770008C2D0E9445278C2F0E94A8278F73F7015C
:103780009081891721F08083DD24D39401C0D12C4E
:103790008C2D0E94A8278F73F7019781891719F044
:1037A000878381E001C080E0D82ADD290E94992723
:1037B000CF5FFFEFEF1AFF0AC730A1F61092E403C4
:1037C000C091E303CC2309F4C4C00E94F0222091ED
:1037D000E1033091E203AC01421B530B9A01909339
:1037E000E2038093E1034F3F510509F018F4452BA4
:1037F00019F102C02FEF30E01092E3031092E003C2
:10380000E091E803F091E903AF01425F5F4F90E080
:1038100030E08081882341F0281718F010829C2F17
:1038200003C0821B80833C2F3196E417F50789F78C
:103830003093E3039093E003DD2309F47BC0E09130
:10384000E803F091E9038091E4039091E303AAEF88
:10385000B3E0AF01425F5F4F64E1E80128813C9132
:10386000321779F0308131110CC060832C9398812C
:103870009227282F30E0292B81E0232B09F480E0C8
:1038800091E0319611960F5F1F4FE417F50729F766
:103890008093E4039093E303C091E4032091C30574
:1038A0008091E6039091E7032223C9F1892B31F43B
:1038B00025982D9826982E9827982F988091E60382
:1038C0009091E7039170892B79F48091E503882327
:1038D00019F026982E9802C0269A2E9A9091E50308
:1038E00081E089278093E5038091E6039091E703C7
:1038F0008130984750F01092C305809128040E94AF
:10390000B6251092E7031092E6038091E6039091AA
:10391000E70301969093E7038093E6031EC0892B8B
:10392000E1F01092E7031092E603809128040E94D0
:10393000B62513C081E09091E003992309F4ACCF40
:1039400081117DCF0E94F0229093E2038093E103E6
:1039500076CFD111F7CF80E0EECF8C2FCDB7DEB789
:10396000E8E00C947D31ACE5B0E0E9EBFCE10C94CF
:10397000593185B7806885BF85B7806885BF84B7B2
:10398000877F84BF0FB6F894A89580916000886106
:1039900080936000109260000FBE90E080E80FB648
:1039A000F89480936100909361000FBE88E896E1DF
:1039B00090936302809362020E94950E0E94B40E5F
:1039C0008091E20084608093E20078948091C60543
:1039D0008823A1F01091E9001F709091EC00892FCD
:1039E000817090FD80E8182B1092E9008091E8002A
:1039F00083FD0E947F0B1F701093E90082E084BD5D
:103A000093E095BD9AEF97BD80936E000E945E266D
:103A100090E090931801809317010E9499270E94CB
:103A2000DF27EAEEF3E0AAEFB3E011921D9223E064
:103A3000E83FF207D1F78EE090E00E947034809367
:103A4000E8039093E903FC010E961192E817F90739
:103A5000E1F789EA8093800089E0809381002498CF
:103A60002C983F988AB18F7C8AB96E98479A8BB10F
:103A700080638BB9769A8FE090E00E940B3260935E
:103A8000290470932A0480932B0490932C0467706C
:103A90003FEF639FB0011124759567957595679504
:103AA0007727709389006093880070938B006093F0
:103AB0008A0070938D0060938C000E94D52680E070
:103AC00090E00E941132883E9E4F11F00E948218B1
:103AD00082E090E00E9403328093080484E090E04A
:103AE0000E940332182F82E290E00E940332212FBD
:103AF00030E0382B30936A022093690283E090E033
:103B00000E9403320E940F2D809128040E94B62546
:103B10000E940A240E94FD230E94FD238091C70574
:103B200081608093C7058BE091E090938D05809331
:103B30008C0578E1672E712C5524539444244394CA
:103B40008091C605853009F071C050E4F52E63E020
:103B5000E62E00E112E18091C605853009F05EC0D5
:103B60008091C605843009F436C00E9428248091D3
:103B70002D0481110DC00E94DA1010921A0180915B
:103B8000C8058370809319010E943921E0922001B9
:103B900040922D04109290050FB6F894A89560926B
:103BA00060000FBEF092600083B7817F846083BFA6
:103BB00083B7816083BF7894889583B78E7F83BFF6
:103BC0000FB6F894A895809160008861809360009A
:103BD000109260000FBE80919302882309F4BBCF3E
:103BE0000E945E2690E090931801809317010E9436
:103BF00099270E94DF27EAEFF3E0119284E0E83092
:103C0000F807D9F70E948D1BEAEFF3E0819181114B
:103C100077C294E0E830F907C9F79DCF10926F02A0
:103C20000E944B2D0E94792310922D040E948D1B1F
:103C300049E0E42E44E0F42EAAEFB3E0F7019191BD
:103C40008D91892724E0E731F20719F08823B9F331
:103C500032C0811130C00E94F0228C018091F803A3
:103C60009091F9030817190709F46AC08FEF649659
:103C70008FAF649765968FAF659766961FAE669710
:103C80000E94F0228160782F68969FAF8EAF689770
:103C900064964FAD649765965FAD659766966FAD18
:103CA000669768968FAD68970E94EB241093F9038E
:103CB0000093F80345C03AEFC32E33E0D32E10E053
:103CC000F60191906F01F701A080A92481F100E035
:103CD000BB24B3948A2D8B2121F169960FAF69978C
:103CE0006A961FAF6A9791E0892D8B2109F490E0C5
:103CF0006B969FAF6B970E94F0228160782F6D9634
:103D00009FAF8EAF6D9769964FAD69976A965FAD1D
:103D10006A976B966FAD6B976D968FAD6D970E949E
:103D2000EB240F5FBB0C0630A9F6F70190821F5FF2
:103D3000FFEFEF1AFF0A1E3009F0C2CF0E94E42203
:103D40000E94282485E0E9E9F5E0DE011196019062
:103D50000D928A95E1F710929A0510929B051092A8
:103D60009C0510929D051A81111104C08B81882336
:103D700009F450C080919705909198050E943F10DA
:103D80009C0190919305992309F4D2C12531310505
:103D900008F440C09F3F19F09F5F90939305112353
:103DA00061F00E94662B111614F491E001C09FEFA0
:103DB000899F802D112480939A051B81112361F026
:103DC0000E94662B111614F491E001C09FEF899FA9
:103DD000802D112480939B0530919A053323D1F0D7
:103DE00020919B052223B1F045EB3403C00111243F
:103DF000992319F090939A0502C050929A0535EBD9
:103E00002303C0011124992319F090939B0502C04C
:103E100050929B051C81111104C08D81882309F4E7
:103E200050C080919505909196050E943F109C018D
:103E300090919205992309F47FC12531310508F449
:103E400040C09F3F19F09F5F90939205112361F04E
:103E50000E94462B111614F491E001C09FEF899F38
:103E6000802D112480939C051D81112361F00E94F7
:103E7000462B111614F491E001C09FEF899F802D0D
